:03000000022AB918
:0C2AB90078FFE4F6D8FD758153022B0075
:100EB10020000A3C2E2E2E3E004950436F6E6E6577
:100EC10063745245510A004950436F6E6E656374F5
:100ED100000A49504E6F41434B210A003E432C56B4
:100EE1002C43432CC0E4E0EFF2E5F020D1E8EDEA39
:100EF100EEEC49500A003E432C4D41432C25303243
:100F010062583A25303262583A25303262583A25D1
:100F1100303262583A25303262583A2530326258BE
:100F21002C4D414320E0E4F0E5F10A003E432C560C
:100F310045522C20332E3220EEF2202573202573CA
:100F41002CC2E5F0F1E8FF20495020ECEEE4F3EB90
:100F5100FF0A0041756720323020323030380030CE
:100F6100373A35323A3436003E432C4C442C5052F9
:100F71004F473A2020202020202020202020202000
:100F81002020202020202020202020202020202060
:100F91002020202020202020202020202020202050
:100FA1002020202020202020202020202020202040
:100FB10020202020202020202CC4E0F2E020EFF08F
:100FC100EEF8E8E2EAE828F4E0E9EB290A003E2A33
:100FD1002C312CCEF1EDEEE2EDFBE520EFE0F0E07F
:100FE100ECE5F2F0FB20F1E5F2E5E2EEE3EE20E8DC
:100FF100EDF2E5F0F4E5E9F1E00A003E412C413083
:10100100312C2562752E2562752E2562752E25627D
:10101100752C495020E0E4F0E5F120E0E4E0EFF246
:10102100E5F0E00A003E412C4130322C2562752E5C
:101031002562752E2562752E2562752C495020E09A
:10104100E4F0E5F120EEF1ED2E20F1E5F0E2E5F03E
:10105100E00A003E412C4130332C2562752E256279
:10106100752E2562752E2562752C495020E0E4F01D
:10107100E5F120F0E5E72E20F1E5F0E2E5F0E00A08
:10108100003E412C4130342C2562752E2562752E8F
:101091002562752E2562752CCCE0F1EAE020F1E5A0
:1010A100F2E80A003E412C4130352C2562752E258F
:1010B10062752E2562752E2562752CD8EBFEE70A26
:1010C100003E2A2C312CC4EEEF2E20EFE0F0E0ECB4
:1010D100E5F2F0FB20F1E5F2E5E2EEE3EE20E8EDEA
:1010E100F2E5F0F4E5E9F1E00A003E422C5330313B
:1010F1002C2562752CC6E4E0F2FC20E7E0EFF0EE6F
:10110100F1E020F1EEE5E4E8EDE5EDE8FF20EEF2B7
:1011110020F1E5F0E2E5F0E00A003E422C533032E6
:101121002C2562752CCEE1ECE5ED20F120F1E5F006
:10113100E2E5F0EEEC20E1E5E720EAE2E8F2E0EDBD
:10114100F6E8E90A003E422C5330332C2562752C17
:10115100CFE5F0E5E7E0EFF3F1EA20EFF0E820EF8B
:10116100EEF2E5F0E520F1E2FFE7E820F120F1E51C
:10117100F0E2E5F0EEEC0A003E454E440A000A4476
:10118100756D7058202020202030302030312030E3
:101191003220303320303420303520303620303783
:1011A1002030382030392030412030422030432057
:1011B1003044203045203046000A3A003A20000AE7
:1011C100000A44756D7044202020202030302030EA
:1011D1003120303220303320303420303520303649
:1011E1002030372030382030392030412030422023
:1011F1003043203044203045203046004572722073
:101201006B657900526420656570726F6D0A0052DA
:1012110064204D454D0A00526420436F64650A0005
:10122100577269746520436F64650A00446562758D
:10123100674950204F4E0A00446562756749502046
:101241004F46460A00446562756755736572204FC3
:101251006E0A00446562756755736572204F464694
:101261000A0044656275674D7367204F6E0A00443A
:10127100656275674D7367204F46460A00436F6E7E
:10128100666967206C6F636B210A00577220656580
:1012910070726F6D0A00205361766520656570720A
:1012A1006F6D210A00457272204D414321004C6F40
:1012B10061643E3E002A003C4130313D003C4130FA
:1012C100323D003C4130333D003C4130343D003C37
:1012D1004130353D003C21003C5330313D003C5311
:1012E10030323D003C5330333D003C5330353D00FE
:0612F1003C5330363D00C5
:06331000010B00010900A1
:10334600C28E438910758BFF758DB7D2ABD28E2294
:03001B0002290CAB
:10290C00C0E0C083C082C0D0C28E758BFF758DB7FE
:10291C0020060675A61E75A6E10509D202E50B6018
:10292C0002050BE50AD394014002150A050EE50ECB
:10293C00540F7048D20EE50E543F7012D2009066C0
:10294C008BE0600A04F0E0D394B44002D2069066A7
:10295C0086E0600204F0906104E0600214F090667E
:10296C008CE0D394014003E014F0300502050CE533
:10297C000DD394644004D2068002050DE508D3946F
:10298C000140021508D28ED0D0D082D083D0E03254
:10085300C2AFC291C290D2B5C20B7D027C007F07AA
:100863001232F38F24E524646060097D017F6012F6
:10087300328ED20BE4FDFC7F0B1232F38F24E5247E
:1008830030E6097D04E4FF1232B2D20B7D017C0015
:100893007F071232F38F24E5247008FD7FFF1232A5
:1008A3008ED20B300B03126000C288C2A8C2AA7595
:1008B3008900122DE190633EE0B4FA06A3E064CE12
:1008C300607BE4F52474362524F582E43463F583F0
:1008D300E4F00524E524B443EC90633E74FAF0A3FA
:1008E30074CEF0A374CCF0906344740AF0E4A3F0E4
:1008F300A304F0A3F090633A74FFF0A3F0A3F0E431
:10090300A3F0906355740AF0E4F524E5242401FF71
:10091300E433FE74362524F582E43463F583E0FD85
:1009230012326A0524E524C3944340DFE4F5A77536
:10093300A61E75A6E1907FF0F0A3F080FE906349B8
:100943007403F0A374CCF0E4906348F012262AC237
:10095300B51230DCC206123083D20BC20DC20C902A
:1009630065767408F09062B47424F0E4A3F09063A5
:100973003EE09062B6F090633FE09062B7F0906320
:1009830040E09062B8F0906341E09062B9F0906308
:1009930042E09062BAF0906343E09062BBF0750A64
:1009A30001E4906577F0C207C208C209C20A200BAE
:1009B30018AF24FE7D03122549E4FF12285C7E0E46
:1009C3007FB1E4FBFDFC12225690668BE06003745A
:1009D30001F0E4906104F0F50C906575F0F50D12EB
:1009E300334675A70775A61E75A6E1D2AFE4F50DCC
:1009F300906104E0700312323B90668CE0B4011105
:100A03009080007410F0E490668CF0D20BC20CC29C
:100A13000D908008E0F52430E405D2077410F0E56A
:100A23002430E508D2099080087420F0E52430E6EC
:100A330008D2089080087440F0E50CC39403401971
:100A4300908002E4F0908001F0908000F0E50C9437
:100A5300064006E4F50C1230839080A0E070031288
:100A63002E5F9080B8E07003122ED99080D0E07092
:100A730003123027908000E0701330071012235DBB
:100A8300906331EFF0D3940040031200269080026C
:100A9300E07006908000E06005D2050209F0C2050F
:100AA300E4F50C906104E060030209F0200B12905E
:100AB3006578E0600C7E0E7FB3122461E490657864
:100AC300F03009121220E5906331EFF0D394004027
:100AD30005E0FF120022200803020C59121F5E904A
:100AE3006331EFF070030209F0906375E054BF24A3
:100AF3007F7003020BC2147003020B9A240260037B
:100B0300020BFB200B077E0E7FBA122461200F031A
:100B1300020C5990634DE07006906351E06067905A
:100B23006682E0FF90634DE0B50724906683E0FEA4
:100B330090634EE0B50618906684E0FE90634FE044
:100B4300B5060C906685E0FE906350E06E603790CA
:100B53006351E06F6003020C59906683E0FF90637A
:100B630052E06F6003020C59906684E0FF90635378
:100B7300E06F6003020C59906685E0FF906354E0D8
:100B83006F6003020C59C2039065777401F012334E
:100B930068750A01020C5990668BE060037401F0DA
:100BA30090667AE0FF906377E06F6003020C5990E0
:100BB300667AE004F0E4F50A906575F0020C5930AA
:100BC3000303020C59906344E070030209F090633D
:100BD30055740AF0123361D203E4F50A906575F097
:100BE30090668604F0E4906679F0A3F0200B677EAC
:100BF3000E7FC8122461805E90668BE060037401EF
:100C0300F0300352906375E020E74B906377E0FF89
:100C1300906679E0FE6F600D906681E07007EE14D8
:100C23006F70338013906679E004F0906331E0FFD6
:100C3300D3940440031227A99060007482F0A37434
:100C430001F0906377E0906002F07E607F007D03A7
:100C5300122BCC0209F0200303020D71E50A706820
:100C630012299CEF60237E647F75906476E02404F0
:100C7300FD122BCC906681E07009906355E0F50A74
:100C83000209F0E4F50A0209F0906686E0D3943C89
:100C93004036906681E0703090668604F01226F448
:100CA300E4906475F0A37412F090667AE090647730
:100CB300F0A374FDF090610563A20190647963A2CF
:100CC300017F12121CAC809E1233568F24E524B48C
:100CD30001159060007483F0E4A3F07E607F007DD3
:100CE30002122BCC0209F0E524D39401401C90603E
:100CF300007483F0A37401F0E52424FEA3F07E6066
:100D03007F007D03122BCC0209F0E50A6401600326
:100D13000209F0906575E004F0200B077E0E7FD288
:100D2300122461906355E0C394C85004E02432F068
:100D3300906575E0C39405400DC203E4906577F0B8
:100D43001233680209F07C667D82906349E0FAA35E
:100D5300E0FB7F02122D5D7E647F75906476E02454
:100D630004FD122BCC906355E0F50A0209F0E50A65
:100D7300640160030209F0906577E014604624FE85
:100D83006042147003020E64240460030209F0E459
:100D9300F50C200F139065777404F0906575E0549B
:100DA30001F0750A010209F09080027410F0E490DA
:100DB3006577F090657504F0750AFA90668274FFA2
:100DC300F00209F0906682E07003020E4E906475A3
:100DD3007480F09064777401F0E4A3F0A304F0A3AB
:100DE3007430F0A3747BF0E4F524747C2524F5823D
:100DF300E43464F583747DF0747D2524F582E43452
:100E030064F583E4F0E5242407906476F07C667D42
:100E130082906349E0FAA3E0FB7F02122D5D7E64BA
:100E23007F75E5242409FD122BCC906681E0601BBD
:100E3300123361D203E4F50A906575F09066860477
:100E4300F0E4906679F0A3F00209F0300F07E49024
:100E53006577F080069065777404F0750AFA0209E5
:100E6300F09080027410F0750A05906575E06401D6
:100E7300FFF09065777401F0EF7019906351E060B3
:100E830013FCA3E0FDA3E0FEA3E0FF906682121A29
:100E93004D0209F090634DE0FCA3E0FDA3E0FEA347
:0D0EA300E0FF906682121A4D0209F080FEF9
:010EB000221F
:10002600906376E0B444047F0180027F009063759C
:10003600E0B447047E0180027E00EE5F604A906372
:100046003EE0906377F090633FE0906378F09063D2
:1000560040E0906379F0906341E090637AF09063BA
:1000660042E090637BF0906343E090637CF09063A2
:10007600767452F09062AE63A2019080A863A201EA
:100086007F06121CAC020849906331E0C394085005
:100096000302085290633EE0FF906377E06F6003CF
:1000A60002085290633FE0FF906378E06F600302BE
:1000B6000852906340E0FF906379E06F60030208A6
:1000C60052906341E0FF90637AE06F60030208524A
:1000D600906342E0FF90637BE06F600302085290FA
:1000E6006343E0FF90637CE06F6003020852906315
:1000F60076E0B444159062AEE0B4FF0E63A20190C0
:1001060080A863A2017F06121CAC90668BE0600398
:100116007401F090668C7464F09063767452F0907B
:100126006375E0646D60030202537BFF7A0E79DD2E
:100136001213597BFF7A0E79F790633EE0F52DA3F3
:10014600E0F52EA3E0F52FA3E0F530A3E0F531A30B
:10015600E0F532121359752DFF752E0F752F547554
:1001660030FF75310F7532607BFF7A0F792D1213D0
:10017600597BFF7A0F79691213597BFF7A0F79CF72
:100186001213597BFF7A0F79FC906344E0F52DA397
:10019600E0F52EA3E0F52FA3E0F5301213597BFF0F
:1001A6007A10792690634DE0F52DA3E0F52EA3E0B5
:1001B600F52FA3E0F5301213597BFF7A107954908E
:1001C6006351E0F52DA3E0F52EA3E0F52FA3E0F5AE
:1001D600301213597BFF7A10798290633AE0F52D3D
:1001E600A3E0F52EA3E0F52FA3E0F5301213597B1B
:1001F600FF7A1079A5906336E0F52DA3E0F52EA3DE
:10020600E0F52FA3E0F5301213597BFF7A1079C27F
:100216001213597BFF7A1079EBA20FE433F52D12F6
:1002260013597BFF7A11791B906681E0F52D121325
:10023600597BFF7A11794690668BE0F52D1213599A
:100246001231337BFF7A1179791213592290637533
:10025600E0644C70737E117F7FFBFDFC122256908A
:10026600637DE0F525A3E0F526E4F528E525906312
:100276007FF0A3E526F07E117FBA7C637D7F7B024B
:10028600122256E4F527852682852583E0FF747FB2
:100296002527F582E43463F583EFF00526E526701D
:1002A6000205250527E527B410DC7E117FBD7C639A
:1002B6007D7F7B101222560528E528C3941040AC9A
:1002C6007E117FC012246122906375E0646C7060B9
:1002D600F5297E117FC2FBFDFC122256E4F528E4C7
:1002E60090637FF0A3E529F07E117FBA7C637D7F62
:1002F6007B02122256E4F527A829E6FF747F2527FC
:10030600F582E43463F583EFF005290527E527B484
:1003160010E67E117FBD7C637D7F7B101222560521
:1003260028E528C3940840B77E117FC012246122B5
:10033600906375E0644B7061F52774672527F58235
:10034600E43463F583E0603274672527F582E4348C
:1003560063F583E0F4602374672527F582E434634C
:10036600F583E0FF747D2527F582E43463F583E0A9
:10037600B507100527E527B408C09061047432F06C
:100386000208499063757421F0300B030208497E18
:10039600117FFD122461020849906375E0B4521A78
:1003A600200B077E127F051224619063757472F02C
:1003B6007E637F757D08122B4522906375E0644944
:1003C6007045200B077E127F1012246190637DE03A
:1003D600F525A3E0F526E4F527852682852583E025
:1003E600FF747F2527F582E43463F583EFF0052655
:1003F600E526700205250527E527B480DC7E637FA8
:10040600757D8A122B4522906375E0644370462001
:100416000B077E127F1812246190637DE0F525A3F9
:10042600E0F526E4F527852682852583E493FF7487
:100436007F2527F582E43463F583EFF00526E5266C
:10044600700205250527E527B480DB7E637F757D71
:100456008A122B4522906375E0645A7053200B076D
:100466007E127F2112246190637DE0F525A3E0F5DD
:10047600267C637D7F7B80AF26AE25123207E4F5AE
:1004860027852682852583E493FF747F2527F582B9
:10049600E43463F583EFF00526E5267002052505AD
:1004A60027E527B480DB7E637F757D8A122B452284
:1004B600906375E06444600302054790637DE0FF46
:1004C60064447003020849EFB4310CC20B7E127FFC
:1004D6002D12246102084990637DE0B4300CD20BE2
:1004E6007E127F3912246102084990637DE0B4329E
:1004F6000CD20C7E127F4612246102084990637D5D
:10050600E0B4330CC20C7E127F54122461020849F7
:1005160090637DE0B4340CD20D7E127F63122461A9
:1005260002084990637DE0B4350CC20D7E127F70DF
:1005360012246102084990637DE0FF12002102083F
:1005460049906104E07013200B077E127F7E12240F
:10055600619063757421F00208499061047432F069
:10056600906375E0FFB45104C2AF80FEEF6457702C
:1005760045200B077E127F8C12246190637EE090EB
:100586006331F0E4F527906331E0FFE527C39F4030
:1005960003020849747F2527F582E43463F583E076
:1005A600FF90637DE0252724ADF582E43461F58371
:1005B600EFF0052780D0906375E064536003020670
:1005C6006A200B077E127F9712246190633EE0FF3C
:1005D6009061B6E06F703C90633FE0FF9061B7E0DA
:1005E6006F7030906340E0FF9061B8E0B5072490EB
:1005F6006341E0FF9061B9E0B50718906342E0FF00
:100606009061BAE0B5070C906343E0FF9061BBE0F0
:100616006F60169063757421F0300B030208497EF3
:10062600127FA6122461020849E4F527E4F50DAF0E
:1006360027FE74AD2527F582E43461F583E0FD12CB
:10064600326A0527E527C394FE40E1C2AFE4907FF6
:10065600F0F0A3F0907FFD74AAF0A374FFF0A374EA
:1006660055F080FE906375E0644F704C90637DE0BA
:10067600F525A3E0F526E5264525700A200B077E1D
:10068600127FAF122461200B077E127FB6122461FF
:10069600E4F527747F2527F582E43463F583E08546
:1006A6002682852583F00526E52670020525052781
:1006B600E527B480DE020849906375E0FFB4452162
:1006C60090637DE0FDA3E0907FF0CDF0A3EDF0C256
:1006D600AF907FFD74AAF0A374FFF0A37455F08069
:1006E600FEEF6465600302085290637DE0FFA3E0BD
:1006F600907FF0CFF0A3EFF0E4F525F526D3907FB9
:10070600F1E09526907FF0E095254020E4F50D2553
:1007160026FFE5253401FE852682852583E0FD1228
:10072600326A0526E5267002052580D17E127FB83D
:10073600122C53EF4E6020120003906344EFF01228
:100746000003906345EFF0120003906346EFF0124A
:100756000003906347EFF07E127FBE122C53EF4EDC
:10076600602012000390634DEFF012000390634E79
:10077600EFF012000390634FEFF012000390635006
:10078600EFF07E127FC4122C53EF4E60201200034E
:10079600906351EFF0120003906352EFF0120003E2
:1007A600906353EFF0120003906354EFF07E127FD4
:1007B600CA122C53EF4E602012000390633AEFF0FA
:1007C60012000390633BEFF012000390633CEFF0DE
:1007D60012000390633DEFF07E127FD0122C53EF90
:1007E6004E6020120003906336EFF0120003906310
:1007F60037EFF0120003906338EFF01200039063B6
:1008060039EFF0E4F527E4F50DE5272401FFE4339D
:10081600FE74362527F582E43463F583E0FD123253
:100826006A0527E527C3944340DCC2AFE4907FF016
:10083600F0A3F0907FFD74AAF0A374FFF0A37455A3
:0C084600F080FE7E637F757D08122B455C
:010852002283
:1031CF00AE07EEC39430400BEED394395005EE2486
:1031DF00D0FF22EEC39461400BEED394665005EE00
:1031EF0024A9FF22EEC39441400BEED39446500521
:0831FF00EE24C9FF22AF0622F5
:10332C009062ADE004F070069062ACE004F0906244
:0A333C00ACE0FEA3E0FF1232D6223F
:1000030012332C1231CFEFC454F0FEC00612332C3E
:080013001231CFD0E02FFF22D3
:102FCA00E49068B1F012332C9068B2EFF0C39430F9
:102FDA004018E0FFD3943950119068B1E02405F508
:102FEA0082E43461F583EFF080119068B1E0240542
:102FFA00F582E43461F583E4F0800C9068B1E00472
:10300A00F0E0D3940840BE752800752900752A009F
:0C301A00E4F52B7B017A617905121DBAE8
:013026002287
:042C53008E2A8F2B0B
:102C57009062ACE4F0A374FFF012332CEF606EF4D3
:102C6700606B852B82852A83E493B507EC752C016D
:102C7700E52B252CF582E4352AF583E4936025902E
:102C870062ADE0252CFF9062ACE03400FE1232D634
:102C9700E52B252CF582E4352AF583E493B5070463
:102CA700052C80CCE52B252CF582E4352AF583E429
:102CB7009370A6E52C24FFFFE434FFFE9062ADE09D
:102CC7002FF09062ACE03EF07E007F0122E4FEFF31
:012CD70022DA
:10262A007E127FD6122C53EF4E70037F01227E1248
:10263A007FD9122C53EF4E600C12332CEF24D02486
:10264A00FF920F8002D20F7E127FDF122C53EF4EC1
:10265A00600C12332CEF24D0906681F08005E49050
:10266A006681F07E127FE5122C53EF4E600C123316
:10267A002CEF24D090668BF08005E490668BF07E78
:10268A00127FEB122C53EF4E600C12332CEF24D036
:10269A0024FF92018002C20190633E63A201906608
:1026AA007B63A2017F06121CAC30013B7E127FF1D4
:1026BA00122C53EF4E603012000390667BEFF0123B
:1026CA00000390667CEFF012000390667DEFF01233
:1026DA00000390667EEFF012000390667FEFF0121F
:0A26EA000003906680EFF07F0022ED
:10318800906576E0C3947C503D906576E0FE04F04F
:1031980074B42EF582E43462F583EFF0BF0A279009
:1031A8006576E0FF04F074B42FF582E43462F583A9
:1031B800E4F0906576E0FF122CD89065767408F0FC
:0731C8009062B5E004F02263
:103083009080007480F090633663A201F583F5822B
:1030930063A2017F08121CAC90633E63A20190807F
:1030A3008863A2017F0A121CAC908092E4F0A3749F
:1030B30032F0A37401F0906348E0FF9080B1F09088
:1030C30080E1EFF09080957455F0A3F09080007448
:0930D30001F090800974F0F02274
:102E5F00908009E04410F09080A0E0706C9080A109
:102E6F007482F09080A874FFF0A3F0A3F0A3F07F1A
:102E7F00039080AEEFF07FCBA3EFF07F039080AC99
:102E8F00EFF0A374CBF09080007402F09068A5125D
:102E9F001A59000000009068A5E0908040F09068FB
:102EAF00A6E0908041F09068A7E0908042F0906893
:102EBF00A8E0908043F0A3E4F0A3F0A3F0A3F09078
:092ECF008018F0A3F0A3F0A3F0B9
:012ED80022D7
:10302700908009E04440F09080D17482F07F039053
:1030370080DEEFF0A374CCF09080027402F0906809
:10304700A9121A59000000009068A9E0908058F072
:103057009068AAE0908059F09068ABE090805AF0B1
:103067009068ACE090805BF0A3E4F0A3F0A3F0A33A
:0B307700F0908030F0A3F0A3F0A3F075
:01308200222B
:102ED900908009E04420F09080B8E0706C9080B94F
:102EE9007482F07F039080C6EFF07FCDA3EFF07F6F
:102EF900039080C4EFF0A374CDF09080C074FFF00C
:102F0900A3F0A3F0A3F09080017402F09068AD12D1
:102F19001A59000000009068ADE090804CF090686C
:102F2900AEE090804DF09068AFE090804EF09068F0
:102F3900B0E090804FF0A3E4F0A3F0A3F0A3F090E9
:092F49008024F0A3F0A3F0A3F032
:012F5200225C
:102D5D008C258D26A907EAFDE975F018A424ACFF92
:102D6D00E5F034808F82F583EDF0EBFDE975F01819
:102D7D00A4FFAEF024ACFBEE34808B82F583A3ED83
:102D8D00F08526828C83E0FDEF24A8FFEE3480FED3
:102D9D008F82F583EDF08526828C83A3E08F828E62
:102DAD0083A3F0852682852583A3A3E0FDE975F035
:102DBD0018A424A8FFE5F03480FE8F82F583A3A329
:102DCD00EDF08526828C83A3A3A3E08F828E83A34F
:042DDD00A3A3F0229A
:062B45008D2AAB07AA0671
:102B4B00908000E030E5079065787401F022906882
:102B5B00A5E0FCA3E0FDA3E0FEA3E0F52E8E2D8DFA
:102B6B002C8C2BAE02AF038E838F8263A201E52DDB
:102B7B00540744C0F583852E8263A201AF2A121D30
:102B8B001EE4FCFDFEE52E252AF52EEE352DF52D4A
:102B9B00ED352CF52CEC352BF52B908040E52BF0FF
:102BAB00A3E52CF0A3E52DF0A3E52EF090800074A7
:102BBB0020F0AF2EAE2DAD2CAC2B9068A5121A4D7C
:012BCB0022E7
:062BCC008D25AB07AA06EF
:102BD200908002E030E5079065787403F0229068F7
:102BE200A9E0FCA3E0FDA3E0FEA3E0F5298E288D79
:102BF200278C26AE02AF038E838F8263A201E52863
:102C0200540744D0F58385298263A201AF25121DA2
:102C12001EE4FCFDFEE5292525F529EE3528F528DB
:102C2200ED3527F527EC3526F526908058E526F078
:102C3200A3E527F0A3E528F0A3E529F0908002742C
:102C420020F0AF29AE28AD27AC269068A9121A4D04
:012C5200225F
:02285C008F25C6
:10285E00908001E030E5099065787402F07F0022E7
:10286E009068ADE0FCA3E0FDA3E0FEA3E0F5298EA9
:10287E00288D278C2690667B63A201E52854074499
:10288E00C8F58385298263A2017F06121D34E529CE
:10289E002406F529E43528F528E43527F527E4350F
:1028AE0026F52690657963A201E528540744C8F5FC
:1028BE008385298263A201AF25121D34E4FCFDFE3F
:1028CE00E5292525F529EE3528F528ED3527F527B7
:1028DE00EC3526F52690804CE526F0A3E527F0A3EF
:1028EE00E528F0A3E529F09080017420F0AF29AE21
:0D28FE0028AD27AC269068AD121A4DAF250D
:01290B0022A9
:10235D009081E0E0F52505250525052505250525B3
:10236D0005250525052505250525908010E0F52871
:10237D00A3E0F529A3E0F52AA3E0F52B9081E1E098
:10238D00F525052505250525052505250525052500
:10239D00052505250525908014E0F52CA3E0F52DE8
:1023AD00A3E0F52EA3E0F52FE52EB52A08E52FB510
:1023BD002B037F0022E4F525E52E540744E0F58339
:1023CD00852F8263A20190637563A2017F08121DA0
:1023DD006490637763A2019062AE63A2017F0612DF
:1023ED001CAC906375E0F526A3E0F527E4F5259088
:1023FD006375E0702AA3E024F8F525E52E54074413
:10240D00E0F583852F8274082582F582E43583F506
:10241D008363A20190637563A201AF25121D64AEA3
:10242D0026E4FCFDE52F2527F52FE52E3EF52EEDB7
:10243D00352DF52DEC352CF52C908014E52CF0A3D5
:10244D00E52DF0A3E52EF0A3E52FF090800074406C
:03245D00F0AF25B8
:012460002259
:101F5E009081E6E0F52505250525052505250525B0
:101F6E0005250525052505250525908028E0F5285C
:101F7E00A3E0F529A3E0F52AA3E0F52B9081E7E095
:101F8E00F525052505250525052505250525052503
:101F9E0005250525052590802CE0F52CA3E0F52DD3
:101FAE00A3E0F52EA3E0F52FE4F525E52EB52A0ADC
:101FBE00E52FB52B05C2080220CAE52E540744F0C2
:101FCE00F583852F8263A20190637563A2017F085A
:101FDE00121D64906375E0F526A3E0F527E527450D
:101FEE002670099080027410F07F0022906682E0C5
:101FFE00FFF46030906377E06F600302209190668B
:10200E0083E0FF906378E06F7079906684E0FF90D4
:10201E006379E06F706D906685E0FF90637AE06F94
:10202E006031805F906377E0906682F0906378E035
:10203E00906683F0906379E0906684F090637AE026
:10204E00906685F090637BE0FFA3E0906349CFF04C
:10205E00A3EFF0906375E0702AA3E024F8F525E570
:10206E002E540744F0F583852F8274082582F5825D
:10207E00E43583F58363A20190637563A201AF25F6
:10208E00121D64AE26E4FCFDE52F2527F52FE52E67
:10209E003EF52EED352DF52DEC352CF52CAF2BAE6A
:1020AE002AAD29AC28AB2FAA2EA92DA82CD3121AF3
:1020BE003C40099080027410F07F002290802CE545
:1020CE002CF0A3E52DF0A3E52EF0A3E52FF09080E4
:0620DE00027440F0AF2582
:0120E40022D9
:1020E5009081E3E0F525052505250525052505252B
:1020F5000525052505250525052590801CE0F528E0
:10210500A3E0F529A3E0F52AA3E0F52B9081E4E00F
:10211500F52505250525052505250525052505257A
:10212500052505250525908020E0F52CA3E0F52D56
:10213500A3E0F52EA3E0F52FE4F525E52EB52A0A53
:10214500E52FB52B05C20902223BE52E540744E8CD
:10215500F583852F8263A20190600463A2017F0E3F
:10216500121D7A906004E0F526A3E0F52790600C37
:10217500E0FFF4604A90667BE0FEEF6E7079A3E0C5
:10218500FF90600DE06F706F90667DE0FF90600ED0
:10219500E06F706390667EE0FF90600FE06F7057B0
:1021A50090667FE0FF906010E06F704B906680E076
:1021B500FF906011E06F703FE4906013F08008902D
:1021C500601374FFF0D2D9906004E0702AA3E02474
:1021D500F2F525E52E540744E8F583852F82740E24
:1021E5002582F582E43583F58363A201906004635B
:1021F500A201AF25121D7AAE26E4FCFDE52F2527A9
:10220500F52FE52E3EF52EED352DF52DEC352CF57E
:102215002CAF2BAE2AAD29AC28AB2FAA2EA92DA801
:102225002CD3121A3C5006E52745267009908001EB
:102235007410F07F0022908020E52CF0A3E52DF0AE
:10224500A3E52EF0A3E52FF09080017440F0AF25B3
:012255002266
:042461008E2A8F2B05
:10246500908000E030E5079065787401F02290686F
:10247500A5E0FCA3E0FDA3E0FEA3E0F5318E308DE1
:102485002F8C2EE531FFE5305407FEE42FF52DEEB8
:1024950034C0F52C852D82F5837423F0052DE52DAB
:1024A5007002052C532CC7F582852C83740AF00520
:1024B5002DE52D7002052C532CC790633E63A201B8
:1024C500852C83852D8263A2017F06121D1E74064D
:1024D500252DF52DE4352CF52C852A83852B826356
:1024E500A201852C83852D8263A201121D02E4FCC5
:1024F500FDFE9068A5E0F8A3E0F9A3E0FAA3E02FBC
:10250500FFEE3AFEED39FDEC38FCEF2408FFE43E22
:10251500FEE43DFDE43CFC9068A5121A4D9068A5CB
:10252500E0908040F09068A6E0908041F09068A728
:10253500E0908042F09068A8E0908043F0908000A1
:032545007420F00F
:012548002270
:0A2256008E2A8F2B8C2C8D2D8B2EE1
:10226000908000E030E5079065787401F022906876
:10227000A5E0FCA3E0FDA3E0FEA3E0F5348E338DE2
:10228000328C31E534FFE5335407FEE42FF530EEB0
:1022900034C0F52F853082F5837423F00530E530A6
:1022A0007002052F532FC7F582852F83740AF0051E
:1022B00030E5307002052F532FC790633E63A201B3
:1022C000852F8385308263A2017F06121D1E74064E
:1022D0002530F530E4352FF52F852A83852B826351
:1022E000A201852F8385308263A201121D028F35E2
:1022F000EF2530F530E4352FF52FE52E6017852CCE
:1023000083852D8263A201852F8385308263A2019C
:10231000AF2E121D1EE5352408252EF52EFFE4FCF8
:10232000FDFEE5342FF534EE3533F533ED3532F57A
:1023300032EC3531F531908040E531F0A3E532F0F3
:10234000A3E533F0A3E534F09080007420F0AF34BF
:0C235000AE33AD32AC319068A5121A4DCE
:01235C00225E
:022CD8008F3E2D
:102CDA00908000E030E5079065787401F0229068F2
:102CEA00A5E0FCA3E0FDA3E0FEA3E0F5428E418D42
:102CFA00408C3FE542FFE5415407FEE42FFFEE34E6
:102D0A00C09062B463A201F5838F8263A201AF3ED1
:102D1A00121D1EE4FCFDFEE542253EF542EE35415C
:102D2A00F541ED3540F540EC353FF53F908040E503
:102D3A003FF0A3E540F0A3E541F0A3E542F090801F
:102D4A00007420F0AF42AE41AD40AC3F9068A5128E
:022D5A001A4D10
:012D5C002254
:062549008E258F26AB0574
:10254F00908000E030E5079065787401F022906884
:10255F00A5E0FCA3E0FDA3E0FEA3E0F52C8E2B8D00
:10256F002A8C29E52CFFE52B5407FEE42FF528EEE6
:10257F0034C0F527852882F5837423F00528E528D4
:10258F00700205275327C7F582852783EBF00528AF
:10259F00E5287002052790633E63A2018527838596
:1025AF00288263A2017F06121D1E74062528F528B6
:1025BF00E43527F5275327C7E52585288285278307
:1025CF00F00528E528700205275327C7F5828527D0
:1025DF0083E526F00528E528700205275327C7E570
:1025EF002C240AF52CE4352BF52BE4352AF52AE4B7
:1025FF003529F529908040E529F0A3E52AF0A3E5D8
:10260F002BF0A3E52CF09080007420F0AF2CAE2BB4
:0A261F00AD2AAC299068A5121A4DEF
:01262900228E
:1032D600A2AF9210C2AF438E2075D2028F828E8328
:0C32E600E0FFE4F5D2538EDFA21092AF9F
:0132F20022B9
:10326A00E5D220E0FBA2AF9210C2AF43D2028F8216
:10327A008E83EDF075D25063D250A21092AFE5D290
:03328A0020E0FB46
:01328D00221E
:102DE100E4FDED2401FFE433FE1232D674362DF5F5
:102DF10082E43463F583EFF00DBD3FE6E4FDED249D
:102E01007FFFE433FE1232D6742D2DF582E4346156
:102E1100F583EFF0742D2DF582E43461F583E070D4
:102E21001B742D2DF582E43461F5837420F0742E2A
:102E31002DF582E43461F583E4F080040DBD80BE9C
:102E4100E49061ACF0FDEDFF7E001232D674AD2D41
:0D2E5100F582E43461F583EFF00DBDFEE97C
:012E5E002251
:023207008B2A10
:10320900A2AF9210C2AF85A22B53A2FE8E838F82EA
:1032190005A28C838D827409121DA8E52A53A2FE8A
:1032290043A220121DAA53A2DF852BA2A21092AF9E
:01323900FF95
:01323A002271
:1032F300A2AF9210C2AF8C838D82EF121DA843A29E
:0C33030020121DAA53A2DFA21092AFFFFF
:01330F00229B
:02328E008F258A
:10329000A2AF9210C2AFE4F5838D827406121DA80E
:1032A000E52543A220121DAA53A2DFA21092AF7FF0
:0132B000011C
:0132B10022FA
:0232B2008F2566
:1032B400A2AF9210C2AFE4F5838D82740A121DA8E6
:1032C400E52543A220121DAA53A2DFA21092AF7FCC
:0132D40001F8
:0132D50022D6
:101BD100A907E7FFA805EF93C3966008403B74FC93
:101BE1002FFF80F00F08EF93C3966008402B74FB22
:101BF1002FFF80E00F08EF93C3966008401B74FA33
:101C01002FFF80D00F08EF93D3966008400B74F933
:101C11002FFF80C01F1F1F1F1FEF54FEF80303F784
:101C2100E893FC08E893FD08E893FE08E893FF2297
:101C310009E993C39D6008402974FB29F980F109E2
:101C4100E993C39E6008401A74FA29F980E209E910
:101C510093D39F6008400B74F929F980D31919199E
:101C61001919E9C313C313FF22740093F8ECC39845
:101C71004024701F740193F8EDC3984019701474D7
:0E1C81000293F8EEC398400E7009740393F8B6
:101C8F00EFC39840037F00227F0122EDF8E6F008B2
:101C9F00A3DFFA22EDF8E0F608A3DFFA22E0A36350
:101CAF00A201F0A363A201DFF475A2002263A201D7
:101CBF00F0A363A20122E0A363A201F0A363A20138
:101CCF00E0A363A201F0A363A201E463A201F0A366
:101CDF0063A201DFE175A20022E0A363A2016DFE02
:101CEF00936CFDEE058393FC158363A201DFEA7508
:101CFF00A200227F00E493A363A201F00F600CA364
:101D0F00E583C2E3F58363A20180EA75A20022E0B6
:101D1F00A363A201F0A3E583C2E3F58363A201DF0E
:101D2F00EE75A20022E0A363A201F0A3E583C2E453
:101D3F00D2E3F58363A201DFEC75A20022E0A36377
:101D4F00A201F0A3E58344F8C2E5F58363A201DFA6
:101D5F00EC75A20022E583C2E3F583E0A363A20141
:101D6F00F0A363A201DFEE75A20022E583C2E4D2E5
:0A1D7F00E3F583E0A363A201F0A3E3
:101D890063A201DFEC75A20022E58344F8F583E044
:101D9900A363A201F0A363A201DFEE75A20022F9F9
:101DA90022C002C004C00612FFF0D006D004D0023F
:011DB9002207
:101653003E2A2C312CCFE0F0E0ECE5F2F0FB20EC5D
:10166300E0E3E8F1F2F0E0EBFCEDEEE3EE20EFEE89
:10167300F0F2E00A003E4C2C4930312C256C752CDD
:10168300D1EAEEF0EEF1F2FC20EEE1ECE5EDE02C38
:1016930035302C3130302C3330302C3630302C3147
:1016A3003230302C323430302C343830302C393620
:1016B30030302C31393230302C33383430302C3513
:1016C300373630302C3131353230300A003E532C2E
:1016D3004930332C2562752CC7E0E4E5F0E6EAE0F7
:1016E30020F1F2E0F0F2E020EFE5F0E5E4E0F7E8E6
:1016F300282A3130ECF1290A003E532C4930342C8E
:101703002562752CCFE0F3E7E020EFE5F0E5E4E0B8
:10171300F7E820EFE0EAE5F2EEE2282A3130ECF1D7
:10172300290A003C21003C4930313D003C4930331B
:101733003D003C4930343D000AC1F3F4E5F020E7B5
:10174300E0EDFFF221000A4F55543E000A3C002011
:10175300212121435243204552523A20000089124D
:101763009B24AD36BF48C15AD36CE57EF7810893FD
:101773001AA52CB73EC940DB52ED64FF76028B10ED
:101783009926AF34BD4AC358D16EE77CF5830A91DD
:1017930018A72EB53CCB42D950EF66FD74048D16C5
:1017A3009F20A932BB4CC55ED768E17AF3850C97BD
:1017B3001EA128B33ACD44DF56E960FB72068F14AD
:1017C3009D22AB30B94EC75CD56AE378F1870E959D
:1017D3001CA32AB138CF46DD54EB62F97008811A95
:1017E300932CA53EB740C952DB64ED76FF89009B7D
:1017F30012AD24BF36C148D35AE56CF77E0A83186D
:10180300912EA73CB542CB50D966EF74FD8B02995C
:1018130010AF26BD34C34AD158E76EF57C0C851E44
:101823009728A13AB344CD56DF60E972FB8D049F3C
:1018330016A920BB32C54CD75EE168F37A0E871C2C
:10184300952AA338B146CF54DD62EB70F98F069D1C
:1018530014AB22B930C74ED55CE36AF1780011238B
:1018630032465765748C9DAFBECADBE9F81001336D
:1018730022564775649C8DBFAEDACBF9E82130025E
:101883001367764455ADBC8E9FEBFAC8D93120124D
:101893000377665445BDAC9E8FFBEAD8C9425361BA
:1018A3007004152736CEDFEDFC8899ABBA5243712D
:1018B3006014053726DECFFDEC9889BBAA6372401E
:1018C3005125340617EFFECCDDA9B88A9B7362500D
:1018D3004135241607FFEEDCCDB9A89A8B8495A772
:1018E300B6C2D3E1F008192B3A4E5F6D7C9485B7ED
:1018F300A6D2C3F1E018093B2A5E4F7D6CA5B486DE
:1019030097E3F2C0D129380A1B6F7E4C5DB5A496CC
:1019130087F3E2D0C139281A0B7F6E5C4DC6D7E539
:10192300F48091A3B24A5B69780C1D2F3ED6C7F5AC
:10193300E49081B3A25A4B79681C0D3F2EE7F6C49D
:10194300D5A1B082936B7A48592D3C0E1FF7E6D48C
:0D195300C5B1A092837B6A58493D2C1E0F40
:1033160052668D0000000000000000000000000062
:053326000000000000A2
:0100210022BC
:03002300022A2B83
:0B2A2B00C0E0C083C082C0D075D0188E
:102A360030984BC298750B01AF99E543700EEF6461
:102A460055703BF54A754301D2918032E553702E9D
:102A5600749F254AF582E43466F583EFF0E54AB4BF
:102A66000104EF04F544E54A600AB5440F04F55342
:102A7600C2918008EF64556003754300054A30999A
:102A860029301A24D290E551B5490DC21AD21CC27A
:102A960090D2968545088010749F2551F582E434BE
:0A2AA60067F583E0F5990551C29928
:092AB000D0D0D082D083D0E032F6
:103133007BFF7A16795312135990689FE0FEA3E040
:10314300FFC3E49FFFE49EFEAB07FA3395E0F9F873
:103153007F007E8C7D0A7C0012199C8F308E2F8D10
:103163002E8C2D7BFF7A1679781213597BFF7A16F2
:1031730079D085462D1213597BFF7A1679FC854544
:053183002D121359227A
:102F53007E177F26122C53EF4E70037F01227E17BC
:102F63007F29122C53EF4E6023122FCAA804A90500
:102F7300AA06AB077F007E8C7D0A7C0012199C1287
:102F83001A2E90689FEEF0A3EFF0800A90689F746A
:102F9300FFF0A374B8F07E177F2F122C53EF4E600F
:102FA30009122FCAEF04F5468003E4F5467E177F26
:102FB30035122C53EF4E6009122FCAEF04F54580EA
:072FC30003E4F5457F002245
:1030DC00C21AC21CE4F543F551F549F54AF50BC289
:1030EC0019755209122F53D296C2ADE4F5C9D2CD3F
:1030FC00D2CCC2C9C2CAF5CDF5CC90689FE0F5CB55
:10310C00A3E0F5CA85CBCD85CACCE4F598D29E4315
:10311C008740C29FC2ACC298C29975B81075B710DF
:07312C00D2CAD29CD2AC22F2
:0100220022BB
:1026F400E4FF0F2405F582E43461F583E552F00F1D
:1027040074052401F582E43461F583E4F07C667D8C
:1027140092FEED1DAA0470011CF5828A83E0FBAAD7
:10272400070F74052AF582E43461F583EBF00EBEDD
:1027340004E07C667D96E4FEED1DAA0470011CF5A0
:10274400828A83E0FBAA070F74052AF582E43461C8
:10275400F583EBF00EBE04E07C667D9AE4FEED1D8D
:10276400AA0470011CF5828A83E0FBAA070F740592
:102774002AF582E43461F583EBF00EBE04E07C6656
:102784007D9EE4FEED1DAA0470011CF5828A83E09F
:10279400FBAA070F74052AF582E43461F583EBF094
:0427A4000EBE04E081
:0127A800220E
:03001E00D2992252
:07336100D2CAD29CD2AC22BB
:1027A9008F25301A0E300B0302285B7E177F3B12F0
:1027B900246122906378E0F5527F797583630582FD
:1027C90063A2019067A263A201E52524FCFF121C04
:1027D900AC90679F7455F0A3F0E52524FEA3F0E5BE
:1027E9002504F549E4F54DF54EE52524FCF5507F22
:1027F900A2758367058263A20190176063A201AF86
:1028090050AE4FAD4EAC4D121CE88F508E4F8D4ED1
:102819008C4D749D2549F582E43467F583E54EF0C6
:10282900749E2549F582E43467F583E54DF0E4F5B6
:1028390051D21AC296E5462508F508700312001E02
:10284900200B0D7E177F497C677D9FAB491222566D
:03285900C21C227C
:10299C00E5537002FF22E55324FEF5259066A163F2
:1029AC00A20190647963A201AF25121CACE4F5433B
:1029BC00F553906475F0E52524FEA3F090667AE05B
:1029CC00906477F0A37419F0E4F54DF54E8525501D
:1029DC007F79758364058263A20190176063A201FD
:1029EC00AF50AE4FAD4EAC4D121CE88F508E4F8D8C
:1029FC004E8C4D200B0D7E177F4F7C647D79AB2563
:102A0C00122256E54E454D6013200B0D7E177F525A
:0E2A1C007C007D4D7B021222567F00227F013E
:012A2A002289
:013368002242
:10323B00300004C2000547300E04C20E054BE508F2
:10324B00B40109E4F508301A0312001E301A0CE51C
:0F325B0047D394144008C21AD21C22E4F547222C
:0B335600301C05C21C7F01227F0022FA
:102AC500020853E493A3F8E493A34003F68001F2CC
:102AD50008DFF48029E493A3F85407240CC8C33312
:102AE500C4540F4420C8834004F456800146F6DFE1
:102AF500E4800B0102040810204080903310E47E2E
:102B0500019360BCA3FF543F30E509541FFEE493D5
:102B1500A360010ECF54C025E060A840B8E493A39C
:102B2500FAE493A3F8E493A3C8C582C8CAC583CAC7
:102B3500F0A3C8C582C8CAC583CADFE9DEE780BE7F
:01332B0000A1
:1019600075F008758200EF2FFFEE33FECD33CDCC3E
:1019700033CCC58233C5829BED9AEC99E5829840C1
:101980000CF582EE9BFEED9AFDEC99FC0FD5F0D69E
:10199000E4CEFBE4CDFAE4CCF9A88222B800C1B9C8
:1019A0000059BA002DEC8BF084CFCECDFCE5F0CB06
:1019B000F97818EF2FFFEE33FEED33FDEC33FCEB3F
:1019C00033FB10D703994004EB99FB0FD8E5E4F9FA
:1019D000FA227818EF2FFFEE33FEED33FDEC33FCE7
:1019E000C933C910D7059BE99A4007EC9BFCE99ADB
:1019F000F90FD8E0E4C9FAE4CCFB2275F010EF2F20
:101A0000FFEE33FEED33FDCC33CCC833C810D7071F
:101A10009BEC9AE899400AED9BFDEC9AFCE899F85A
:0E1A20000FD5F0DAE4CDFBE4CCFAE4C8F922ED
:0E1A2E00C3E49FFFE49EFEE49DFDE49CFC22C9
:101A3C00EB9FF5F0EA9E42F0E99D42F0E89C45F000
:011A4C002277
:0C1A4D00ECF0A3EDF0A3EEF0A3EFF0220C
:101A5900A8828583F0D083D082121A70121A70126C
:101A69001A70121A70E473E493A3C583C5F0C58391
:101A7900C8C582C8F0A3C583C5F0C583C8C582C8D7
:011A8900223A
:1012F700E539242DF8E6053922782A301702782DAA
:10130700E475F001121B31021A8A2010EB7F2ED2EE
:10131700108018EF540F2490D43440D4FF30140BAE
:10132700EF24BFB41A0050032461FFE53A600215A9
:101337003A053DE53D7002053C30170D782AE47506
:10134700F001121B31EF021AD00231887403D21751
:101357008003E4C217F5398B2A8A2B892CE4F53AE6
:10136700F53CF53DE53A60077F2012133280F575AD
:101377003BFFC211C210C212C213C215C216C21855
:10138700121300FF700D3017057F00121343AF3D96
:10139700AE3C22B4255FC2D5C214121300FF24D07D
:1013A700B40A00501A75F00A783A30D50508B6FF26
:1013B7000106C6A426F620D5047002D21380D924CC
:1013C700CFB41A00EF5004C2E5D214021543D2116C
:1013D70080C6D21080C0D21280BCD2D580BAD215B6
:1013E70080B47F201213322012077401B53A0040EF
:1013F700F11212F7FF12133202136BD218D21680B2
:10140700951212F7FB1212F7FA1212F7F94A4B70FC
:101417000679147A167BFF20122EE53A602A7E00A1
:101427008E82758300121AA360060EEE653B70F07C
:10143700C2D5EBC0E0EAC0E0E9C0E0EE12158AD001
:10144700E0F9D0E0FAD0E0FB121A8AFF60AAEBC0FD
:10145700E0EAC0E0E9C0E0121332D0E02401F9D09D
:10146700E03400FAD0E0FBE53B0460DCD53BD980F3
:10147700877BFF7A157986D212809C791080027952
:1014870008C216C2188008D2D5790A8004790AC220
:10149700D5E53B047002F53BE4FAFDFEFF1212F7B7
:1014A700FC7B082011131212F7FD7B1030100A1273
:1014B70012F7FE1212F7FF7B20EC3382D592D5503C
:1014C70013C3E43010069FFFE49EFEE42011039D42
:1014D700FDE49CFCE4CBF8C211EC700CCFCECDCC74
:1014E700E824F8F870F38017C3EF33FFEE33FEED0F
:1014F70033FDEC33FCEB33FB994002FB0FD8E9EBF0
:10150700301105F8D0E0C448B211C0E00AEC4D4EE6
:101517004F78207B0070C2EAB53B0040BCC0E012A8
:10152700158CD0F0D0E0201104C4C0E0C4B211C0C3
:10153700F012131BD0F0D5F0EB02136B121B9014B3
:10154700085314825813D94C13D54214864F148E5E
:0F15570044148E4913EE431494551478461478B7
:101566004514784716345013DD2D13E12E14042B41
:1015760013E523140220161D2A139D48000013FCB0
:101586003F3F3F00790AA2D5201314301509B91040
:10159600020404B9080104A2D52016025001042051
:1015A60012689212B53A005034C0E07F2030131909
:1015B6007F30A21272167215500F1215E3C212C2B4
:1015C60016C215C2187F30800F301503E9C0E0122D
:1015D6001332301503D0E0F9D0E0B53ACC30151708
:1015E6007F30B9100C1213327F583014077F788081
:1015F60003B908031213323012057F2D0213327F0E
:10160600202018F87F2B2016F322921280CF286E06
:10161600756C6C2900D2111212F73011F8C21178CC
:101626003A30D50108F602139D2D5043495812123F
:10163600F72403B405004001E490162F93121323F8
:0D164600743A121323D213753A0402148271
:101DBA008B258A268927E4F531F530F52FF52EF59E
:101DCA002CF52DE529452A45286012EBC0E0EAC02A
:101DDA00E0E9C0E0AB28AA29A92A121B41AB2505D4
:101DEA0027E527AA267002052614F9121A8AF5325F
:101DFA00C394094007E532D3940D40E1E5326420EB
:101E0A0060DBE532B42D05432D038016E532B42B91
:101E1A0005432D01800C74FF2527F52774FF35260D
:101E2A00F526E52B60046410703FAB25AA26A92786
:101E3A00121A8A64306009E52B702E752B0A8029E4
:101E4A00900001121AA3FF64786004EFB458134398
:101E5A002D01752B1074022527F527E43526F52662
:101E6A008007E52B7003752B08AB250527E527AA04
:101E7A00267002052614F9121A8AF532C3946140B3
:101E8A000AE532D3947A50035332DF74D02532F5FF
:101E9A0032C3940A400CE5329411406D74F925322C
:101EAA00F532E532D3952B5060432D0185313685C5
:101EBA003035852F34852E33AF2B7E00E4FCFDAB05
:101ECA0031AA30A92FA82E121AE2C8ECC8C9EDC946
:101EDA00CAEECACBEFCBE4FCFDFEEB2532F531EEC0
:101EEA003AF530ED39F52FEC38F52EAF31AE30AD8D
:101EFA002FFCAB36AA35A934A833D3121A3C5003A7
:101F0A00021E73432D04021E73E52D20E003E480B4
:101F1A002DE529452A4528601EAB25E52724FFF92A
:101F2A00E52634FFFAEBC0E0EAC0E0E9C0E0AB28FE
:101F3A00AA29A92A121B41E52D30E20774FFFFFEE8
:101F4A00FDFC22E52DAF31AE30AD2FAC2E30E103D2
:041F5A00021A2E2217
:101A8A00BB010689828A83E0225002E722BBFE025A
:091A9A00E32289828A83E493228D
:101AA300BB010CE58229F582E5833AF583E02250F8
:101AB30006E92582F8E622BBFE06E92582F8E22242
:0D1AC300E58229F582E5833AF583E493225C
:101AD000BB010689828A83F0225002F722BBFE01F5
:021AE000F322EF
:101AE200E88FF0A4CC8BF0A42CFCE98EF0A42CFCA3
:101AF2008AF0EDA42CFCEA8EF0A4CDA8F08BF0A421
:101B02002DCC3825F0FDE98FF0A42CCD35F0FCEB7F
:101B12008EF0A4FEA9F0EB8FF0A4CFC5F02ECD3944
:0F1B2200FEE43CFCEAA42DCE35F0FDE43CFC22B1
:101B3100FAE6FB0808E6F925F0F618E6CA3AF622B5
:101B4100BB011A89828A83D0F0D0E0F8D0E0F9D0C5
:101B5100E0FAD0E0FBE8C0E0C0F0021BBF5016E99C
:101B6100F8D083D082D0E0F9D0E0FAD0E0FBC08297
:101B7100C083021BB6BBFE16E9F8D083D082D0E049
:0F1B8100F9D0E0FAD0E0FBC082C083021BC8227B
:101B9000D083D082F8E4937012740193700DA3A3E4
:101BA00093F8740193F5828883E4737402936860F8
:061BB000EFA3A3A380DFF8
:091BB600EBF608EAF608E9F62254
:091BBF00EBF0A3EAF0A3E9F02227
:091BC800EBF208EAF208E9F2224E
:00000001FF
